:1000000000000000000008280000000000000000C0
:10001000283084005830A0008001840AA00B0C28EE
:10002000103095002730960000308E0000308F0091
:10003000013090000B30970007309F008316FF308F
:10004000850083128316CD30860083120C1D26286E
:100050000C116400A914A9182915A91C2911A919A2
:1000600032282911861A3528291123302B02031929
:100070004028A00020092B05A006A01B45284C28DD
:1000800027302A02031C45284C28291D4A28AA0F7C
:100090004A28AB0A29114D28291529192916291D85
:1000A0002912A9182915A91C2911051B582829113D
:1000B000A91A5E280130AC000030AD00A91629193C
:1000C000762800302D0203196C28A00020092D0588
:1000D000A006A01B7128752801302C02031C712872
:1000E0007528AC0F7428AD0A29157A280030AC00A9
:1000F0000030AD0029192917291D29132919842831
:10010000A91F8328291585282911291BA917291F0B
:10011000A913291D90282E189028AF0F9028B00AF7
:1001200029192E14291D2E100030300203199F2882
:10013000A00020093005A006A01BA428A628013095
:100140002F02031CA428A6282911A728291529193C
:10015000A915291DA911A9182915A91C2911851B43
:10016000B2282911291DB8280030AF000030B00096
:10017000A9182915A91C2911AE1029192E15291DF8
:100180002E11AE19C4282E112E1DC728AE14291900
:100190002E15291D2E11051BCE282E112E1DD128FE
:1001A000AE14AE182915AE1C2911291DDB2800300C
:1001B000AF000030B000A9182915A91C2911AE19EB
:1001C000E2282911291DE8280030B1000030B200D2
:1001D000A9182915A91C2911051BEF28291129196E
:1001E0002E16291D2E12A9182915A91C2911291A04
:1001F000FA28291129192917291D2913AE1E0129A9
:100200002911291BAE16291FAE12291D0C292E1BE0
:100210000C29B10F0C29B20A29192E17291D2E13EA
:100220000030320203191B29A00020093205A00664
:10023000A01B2029222901303102031C2029222958
:100240002911232929152919AE17291DAE13A9181B
:100250002915A91C291186182E292911291D45297E
:100260000030340203193B29A00020093405A00600
:10027000A01B4029442963303302031C4029442930
:10028000B30F4329B40A291149290030B3000030C3
:10029000B400291D4F290030B1000030B200A91868
:1002A0002915A91C2911291A56292911291D5C294A
:1002B0000030AA000030AB00A9182915A91C29118B
:1002C00035102919B514291DB510291A6829B5103A
:1002D000B51C6B2935142919B514291DB510AE1993
:1002E0007229B510B51C89290030370203197F29FE
:1002F000A00020093705A006A01B842988296330A7
:100300003602031C84298829B60F8729B70AB5103D
:100310008D290030B6000030B700B51C9029351487
:1003200035182915351C2911291DB0293519B02971
:10033000B80F9B29B90A003039020319A629A00079
:1003400020093905A006A01BAB29AC295130380281
:10035000031CAB29AC29B0290030B8000030B9002B
:1003600029193515291D3511A9182915A91C291177
:100370005030BA000030BB0038083A02031DC529CE
:1003800039083B02031DC529C62929112919AE15B3
:10039000291DAE11A9182915A91C2911B511291952
:1003A0003516291D3512AE1DD6293512A919D929A0
:1003B0003512351EDC29B51529193516291D3512BA
:1003C000051BE3293512351EE629B515B519291582
:1003D000B51D291129198616291D8612A918291556
:1003E000A91C2911B51229193517291D3513861A8B
:1003F000FA293513061EFD293513351F142A00303E
:100400003D0203190A2AA00020093D05A006A01BF1
:100410000F2A132A09303C02031C0F2A132ABC0F8F
:10042000122ABD0A3513182A0030BC000030BD0066
:10043000B51B1E2A0930BE000030BF00B517351BA2
:10044000362A00303F0203192C2AA00020093F055C
:10045000A006A01B312A352A09303E02031C312A8E
:10046000352ABE0F342ABF0A35173A2A0030BE009B
:100470000030BF00351F3D2AB51629193517291D33
:100480003513051B442A3513351F472AB516B51AEF
:100490002915B51E291129190616291D06128A01CA
:1004A0002628FF3FFF3FFF3FFF3FFF3FFF3FFF3F4C
:1004B000FF3FFF3FFF3FFF3FFF3FFF3FFF3FFF3F4C
:1004C000FF3FFF3FFF3FFF3FFF3FFF3FFF3FFF3F3C
:1004D000FF3FFF3FFF3FFF3FFF3FFF3FFF3FFF3F2C
:1004E000FF3FFF3FFF3FFF3FFF3FFF3FFF3FFF3F1C
:02400E00503F21
:10420000FF00FF00FF00FF00FF00FF00FF00FF00B6
:10421000FF00FF00FF00FF00FF00FF00FF00FF00A6
:10422000FF00FF00FF00FF00FF00FF00FF00FF0096
:10423000FF00FF00FF00FF00FF00FF00FF00FF0086
:10424000FF00FF00FF00FF00FF00FF00FF00FF0076
:10425000FF00FF00FF00FF00FF00FF00FF00FF0066
:10426000FF00FF00FF00FF00FF00FF00FF00FF0056
:10427000FF00FF00FF00FF00FF00FF00FF00FF0046
:10428000FF00FF00FF00FF00FF00FF00FF00FF0036
:10429000FF00FF00FF00FF00FF00FF00FF00FF0026
:1042A000FF00FF00FF00FF00FF00FF00FF00FF0016
:1042B000FF00FF00FF00FF00FF00FF00FF00FF0006
:1042C000FF00FF00FF00FF00FF00FF00FF00FF00F6
:1042D000FF00FF00FF00FF00FF00FF00FF00FF00E6
:1042E000FF00FF00FF00FF00FF00FF00FF00FF00D6
:1042F000FF00FF00FF00FF00FF00FF00FF00FF00C6
:00000001FF
